:040000008A15372FF7
:08000800FF00030E8312031335
:10001000B9000A0EBA00040EBB008A150A125C2F42
:100020000330B807B80CB80C7F30B8050000B80B27
:10003000162808003B08C000BF010310C00DBF0D0B
:10004000C00DBF0DC0070318BF0AC0070318BF0AC1
:100050003330C0070318BF0A00303F078A003C084E
:10006000BF004008820000308A000030C000CD3060
:10007000C62800308A000130C0002D30C62800306C
:100080008A000130C0003530C62800308A000130B7
:10009000C0003E30C62800308A000130C000443025
:1000A000C62800308A000130C0004A30C62800301F
:1000B0008A000130C0004E30C62800308A0001306E
:1000C000C0005330C62800308A000130C0005830CC
:1000D000C62800308A000130C0005F30C6280030DA
:1000E0008A000130C0006930C62800308A00013023
:1000F000C0007130C62800308A000130C0007A305C
:10010000C62800308A000130C0008330C628003085
:100110008A000130C0008F30C62800308A000130CC
:10012000C0009B30C62800308A000130C000A730D4
:10013000C62800308A000130C000B030C628003028
:100140008A000130C000BA30C62800308A00013071
:10015000C000C230C62800308A000130C000CB3059
:10016000C62800308A000130C000D630C6280030D2
:100170008A000130C000DD30C62800308A0001301E
:10018000C000E930C6280130C000F430BF070318B2
:10019000C00A40088A003F088200A234D6340234E4
:1001A00002348434D7348634973426340334A63466
:1001B0009534A634D53402341634A634D734A63454
:1001C0009734803404344034103409340034043417
:1001D00015344034203404341E34A434D734263447
:1001E000573496349E34A034D43492349E34A4349C
:1001F000D53424345534A634D4342634433490349E
:100200009C348234C23429344134A034C0342A347A
:10021000623423346234A234D63424345734A334C1
:10022000D63425345734A634953410341C34A234D3
:10023000C234683440346334423449342034243482
:100240000B34C83494342034D03401342034823414
:10025000063448340034803480344A3441344E34D7
:1002600055344134523459340034463445344234E0
:100270005234553441345234593400344D344134BD
:1002800052344334483400344134503452344934C5
:100290004C3400344D344134593400344A345534EC
:1002A0004E34453400344A3455344C3459340034D7
:1002B0004134553447345534533454340034533472
:1002C00045345034543445344D344234453452343A
:1002D00000344F34433454344F3442344534523470
:1002E00000344E344F34563445344D344234453462
:1002F0005234003444344534433445344D3442346C
:1003000045345234003401340034023402340334AE
:100310000234023401340034013400340034013436
:10032000003402340234033403340334023400341E
:1003300001340034003409340934083408340734F3
:100340000734073408340A3409340934093453347F
:100350004534543420345934453441345234003413
:1003600053344534543420344D344F344E345434A3
:100370004834003453344534543420344434413404
:1003800059340034533445345434203448344F34D1
:1003900055345234003453344534543420344D34BD
:1003A00049344E3455345434453400345034523486
:1003B00045345334453454340034533445344C3488
:1003C0004534433454342034543445345334543451
:1003D00000344B3441344234543452344F344E346C
:1003E00049344334533400343034313432343334C8
:1003F0003434353436343734383439344134423493
:1004000043344434453446340034F808031D092A83
:100410000800F930FF3E031D0A2A0000F80B092AE4
:1004200008008312031385100800831203130511BB
:1004300008008312031385140800831203130515A3
:100440000800831203130510080083120313051418
:1004500008000A3083160313B80010200800B608FD
:100460000319342A1922352A11228316B7080319D1
:100470003B2A1D223C2A152229222522292221221B
:1004800029220800292225222922212229220800A6
:10049000B401B201B301B31908000310B20DB00DDD
:1004A000B40D31083402031C572AB4003214B30AC5
:1004B0004B2AB201B401B301B31908000310B40D03
:1004C000B00DB20D31083202031C682AB200341498
:1004D000B30A5C2AA8012708BB002808BC00A80AA8
:1004E0001A20AB0083132618831725088400A50A59
:1004F0000319A60A2B0880008A110A12031D6B2A11
:100500000800A9012708B0000A30B10059223408B8
:10051000A8002808003C03189B2A28083038AA00A5
:10052000831326188317250884002A088000A50A4B
:100530000319A60A9D2A0130A9002708B0000A3035
:10054000B10048223408A80028083038AA008313D4
:1005500026188317250884002A0880002908AA0085
:1005600008002E08B0000A30B10059223408AF004C
:100570002F083038B00083132D1883172C088400FF
:10058000300880002E08B0000A30B100482234083C
:10059000AF00AC0A0319AD0A2F083038B00083133E
:1005A0002D1883172C0884003008800008001122C1
:1005B0001522212229222522292219221D2229221F
:1005C0000800252219221D22292211221522292262
:1005D00021222922080080303405B60080303505FC
:1005E000B7002F2240303405B60040303505B70043
:1005F0002F2220303405B60020303505B7002F22D9
:1006000010303405B60010303505B7002F22083001
:100610003405B60008303505B7002F220430340504
:10062000B60004303505B7002F2202303405B6007D
:1006300002303505B7002F2201303405B6000130F5
:100640003505B7002F224222080083160313A301A9
:100650001130230203180800831283132030840012
:1006600083162308840700308000A30A282B34084F
:10067000B500B6013030350236080318412B031996
:10068000472B35085F3C0318360803194A2BB9017C
:10069000BA016E2B30303502B7003608B800031CA3
:1006A000B803B708B8080310B70DB80D8312510886
:1006B0008316BB003708BC001A20BE00BD018312A0
:1006C00051088316BB0001303707BC008A110A129B
:1006D0001A20BD043D08B9003E08BA003908BB0025
:1006E0003A08BC000800B201B301AF01B001B1018A
:1006F000311A08000310AF0DB00DA50DA60DB20DF7
:10070000B30D28083302031D872B27083202031C70
:10071000902B2708B2022808031CB303B3022F143E
:10072000B10A782BAF01B001B601B701B101311A9E
:1007300008000310B60DB70DA80DA90DAF0DB00D33
:100740002B083002031DA62B2A082F02031CAF2BF7
:100750002A08AF022B08031CB003B0023614B10AFA
:10076000972B83160313981CB12B7A0883129900D8
:10077000080083160313A3010430230203180800A2
:10078000E1222308003A0319CC2B013A0319D12B9B
:10079000033A0319D62BDB2B7030B400B500EB22E3
:1007A000DF2B7230B400B500EB22DF2B7430B400C5
:1007B000B500EB22DF2B7630B400B500EB22230826
:1007C000A4000310A40D8312831320308400831629
:1007D000240884070008B40037233B08AC003C0819
:1007E000AD0083128313203084008316240A84070B
:1007F0000008B4008A110A1237233B08AE003C08F7
:10080000AF0083128313203084000830831624073E
:1008100084070008B4008A110A1237233B08B0008D
:100820003C08B10083128313203084000930831602
:10083000240784070008B4008A110A1237233B08F2
:10084000B2003C08B300B401B5018A110A12EB22D0
:100850006730B400B500EB222D08B4003108B500B4
:10086000EB222F08B4003308B500EB222C08B400AB
:100870003008B500EB222E08B4003208B500EB2298
:10088000D722A30ABC2B83124408013A03196A2C0D
:10089000033A03196E2C013A0319722C073A031913
:1008A000762C013A03197A2C033A03197E2C013A6B
:1008B0000319822C0F3A0319862C013A03198A2C4A
:1008C000033A03198E2C013A0319922C073A0319A3
:1008D000962C992C52088316A400992C5308831641
:1008E000A400992C54088316A400992C550883164B
:1008F000A400992C56088316A400992C5708831637
:10090000A400992C58088316A400992C5908831622
:10091000A400992C5A088316A400992C5B0883160E
:10092000A400992C5C088316A400992C5D088316FA
:10093000A40000308316A60020302307A50003186A
:10094000A60A2408A7006A2208000030A60020306A
:10095000A500831244088316A7008122AA08031960
:10096000B42C0130A400B62C0230A40083128313EF
:100970002030840083162408A40A84075E30800097
:100980000030A60020302407A5000318A60A831211
:1009900043088316A7008122AA080319D12CA40AB0
:1009A000D32CA40AA40A8312831320308400831654
:1009B0002408A40A84075E308000A3080319112DBF
:1009C0000030AD0020302407AC000318AD0A8312BC
:1009D0003C088316A80083123D088316A9006430E2
:1009E000AA00AB0192233608AE00B1220030AD0060
:1009F00020302407AC000318AD0A0230AC070318FE
:100A0000AD0A83123C088316A50083123D088316A5
:100A1000A6006430A700A80173233208AE00B122FB
:100A200008000030AD0020302407AC000318AD0AE8
:100A300083123C088316A50083123D088316A60086
:100A40006430A700A80173233208AE00B122080069
:100A5000003083160313AD002030AC000B30AC0720
:100A60000318AD0A831242088316AE00B1223A3051
:100A70008312AD0000308316AD002030AC000E3084
:100A8000AC070318AD0A831241088316AE00B122E9
:100A90000800831242088316B0000C30B1004822CF
:100AA0003408A400A408031D572D0C30A40024080A
:100AB000093C0318662D0030AD0020302307AC0040
:100AC0000318AD0A2408AE00B122782D83128313D7
:100AD00020308400831623088407203080002408F7
:100AE0003038A50020308400230A840725088000C0
:100AF0008312831320308400023083162307840777
:100B00003A3080000030AD0020302307AC000318DD
:100B1000AD0A0330AC070318AD0A831241088316EF
:100B2000AE00B1220C30831242020318A12D8313B0
:100B3000203084000530831623078407413080006D
:100B4000AA2D8313203084000530831623078407E1
:100B500050308000831283132030840006308316C7
:100B6000230784074D308000080025230030A600AD
:100B70002030A5007908A7006A220800C601C70135
:100B8000C801C901CA01C61A0800361CD52D320891
:100B9000C70733080318330FC80734080318340F86
:100BA000C90735080318350FCA070310B90CB80C6C
:100BB000B70CB60C0310B20DB30DB40DB50DC60ACB
:100BC000C32DBE01C101C2013208BF003308C000FD
:100BD0003E1A0800341CF22D3F08C10740080318D4
:100BE000400FC2070310B50CB40C0310BF0DC00DAD
:100BF000BE0AE82DFE01B001B101B201B30128081F
:100C0000AC002908AD00AE01AF017E1A08002A1C15
:100C1000172E2C08B0072D0803182D0FB1072E082A
:100C200003182E0FB2072F0803182F0FB307031056
:100C3000AB0CAA0C0310AC0DAD0DAE0DAF0DFE0A42
:100C4000052EC601C701C801C901CB01CC01CD01E8
:100C5000CE01CA01CA1A08000310CB0DCC0DCD0D70
:100C6000CE0DBA0DBB0DBC0DBD0DC60DC70DC80D0B
:100C7000C90D41084902031D472E40084802031DC3
:100C8000472E3F084702031D472E3E084602031C1D
:100C9000582E3E08C6023F08031C3F0FC7024008FB
:100CA000031C400FC8024108031C410FC9024B142A
:100CB000CA0A2A2EFC0183137B1883177A08840042
:100CC0007C08FC0A84070008FD0083137918831749
:100CD00078088400F80A0319F90A7D088000031DCA
:100CE0005B2E0800780883160313AC007908AD006A
:100CF0007A08AE00B122B92308008312031344031B
:100D0000FA005F088316BB007A08BC001A20FE00B8
:100D100083125E088316BB007A08BC008A110A128F
:100D20001A20FB00831260088316BB007A08BC00FF
:100D30008A110A121A20FC0002307C07FD0083127F
:100D40004308093C031CFD0A8A110A122523831259
:100D50003C088316A80083123D088316A90064305E
:100D6000AA00AB0192233608A00083123C08831628
:100D7000A50083123D088316A6006430A700A801D1
:100D800073233208A1008312C7080319CB2E013048
:100D90008316A200CE2E46088316A2002208003A2F
:100DA0000319E82E013A0319262F033A0319462F97
:100DB000013A03194B2F073A0319502F013A03192F
:100DC000742F033A0319782F013A03197D2F822FCC
:100DD0007B08A30043240030A60020307C07A50038
:100DE0000318A60A831243088316A70081228312E0
:100DF0004408093A031D0C2F4308093C03180C2F23
:100E000000308316AD0020307D07AC000318AD0A1A
:100E10002108AE00B122822F00308316AD002030B1
:100E20007D07AC000318AD0A2008AE00B1220030E7
:100E3000AD0020307D07AC000318AD0A0230AC07CE
:100E40000318AD0A2108AE00B122822F7B0AA3004D
:100E500043240030AD0020307C07AC000318AD0AFD
:100E60000130AC070318AD0A2008AE00B1220030F3
:100E7000AD0020307C07AC000318AD0A0330AC078E
:100E80000318AD0A2108AE00B122822F04307B077F
:100E9000A3004324822F7E0AA30043242825822F07
:100EA0007E08A3004324831242088316B0000C304E
:100EB000B10048223408F900F908031D612F0C30F5
:100EC000F90083124408093A031D6F2F7908093C81
:100ED00003186F2F0A308316A3004925822F09308B
:100EE0008316A3004925822F0130A300A524822F59
:100EF0000130A300A5242825822FA301A5240930B1
:100F0000A3004925B92308000F307905FA00B12361
:100F1000790E0F391038FA00B1230800D930F900E2
:100F2000831203133108F9070B30FA003208031853
:100F3000320FFA070130FB0033080318330FFB07A9
:100F40000030FC0034080318340FFC0779088316BE
:100F5000BA007A08BB007B08BC007C08BD00BA0D53
:100F6000BB0DBC0DBD0DBA0DBB0DBC0DBD0DFC30D8
:100F7000BA05B130BE003A30BF000230C0000030C8
:100F8000C10021264B08FD004C08FE00B130B20024
:100F90003A30B3000230B4000030B5007D08B6002E
:100FA0007E08B700B801B901BE254708BA00480855
:100FB000BB004908BC004A08BD000330BE003A0827
:100FC000BE070030BF003B0803183B0FBF070030CF
:100FD000C0003C0803183C0FC0070030C1003D08AA
:100FE00003183D0FC107C10CC00CBF0CBE0CC10CD7
:100FF000C00CBF0CBE0C3F30C1053E087902A000FA
:101000007A08A1007B08A2007C08A3003F08031C0B
:101010003F0FA1024008031C400FA2024108031C1D
:10102000410FA3022008B6002108B7002208B8002B
:101030002308B900B60A0319B70A0319B80A031935
:10104000B90AA030B2000F30B300B401B501BE251B
:101050004708BA004808BB004908BC004A08BD0060
:101060000930BE004B30BF001630C0000030C10058
:1010700021264B08A4004C08A500B530B20005306D
:10108000B3002408B4002508B500E1254108B600E6
:101090004208B700B70CB60CB70CB60C3F30B7051A
:1010A000B801B90136082002BA002108BB002208A5
:1010B000BC002308BD003708031C370FBB023808EB
:1010C000031C380FBC023908031C390FBD021F3046
:1010D000A6003A08A6070030A7003B0803183B0FFC
:1010E000A7070030A8003C0803183C0FA8070030F1
:1010F000A9003D0803183D0FA9075030B200B30105
:10110000B401B5012608B6002708B7002808B800C2
:101110002908B900BE254708BA004808BB0049089D
:10112000BC004A08BD008F30BE000930BF00C001BE
:10113000C10121264B08AA004C08AB004D08AC00A9
:101140004E08AD002A08BA002B08BB002C08BC00D2
:101150002D08BD000B30BE00BF01C001C10121261A
:101160004B08AE004C08AF004D08B0004E08B1006F
:1011700031307D02B4007E08B500031CB503643035
:10118000B200B301E1254108B7004208B6002408C7
:10119000B7072508B80036080318B80AB807B90118
:1011A000BA012E083707BB002F08BC003808031807
:1011B000380FBC073B088312BC0083163C0883121F
:1011C000BD0002308316BE002A08BE070030BF00F3
:1011D0002B0803182B0FBF070030C0002C08031882
:1011E0002C0FC0070030C1002D0803182D0FC107B8
:1011F0000C30B200B301B401B5012E08B6002F08BF
:10120000B7003008B8003108B900BE254708BA0059
:101210004808BB004908BC004A08BD003A083E0225
:101220008312C4008F308316B2000930B300B401BA
:10123000B5012A08B6002B08B7002C08B8002D0805
:10124000B900BE254708BA004808BB004908BC00E1
:101250004A08BD005030BE00BF01C001C1012126B7
:101260004B08C2004C08C3004D08C4004E08C5001E
:10127000420826028312C30008006F30831603134E
:10128000A8000130A90083123C088316AA0083122B
:101290003D088316AB008A11FA253008F8003108A2
:1012A000F9003208FA003308FB00A9010930831263
:1012B00044078316A8000318A90A0C30AA00AB0142
:1012C00092233608FE003708B5007E0883123C07DB
:1012D0008316B40083123D088A15031C71298316F6
:1012E000B50A8316B5070730B200B3018A11E125AC
:1012F0004108A0004208A100A201A301A10CA00C7A
:10130000A10CA00C3F30A1051330B2000130B30096
:10131000831244088316B400B501E1254108A800F2
:101320004208A9000930AA00AB0192233608FC004C
:101330003708FD00831243088316A800A901AA01FB
:10134000AB01B630A4002808A4074230A500290844
:101350000318290FA5071A30A6002A0803182A0F18
:10136000A6070030A7002B0803182B0FA70720089B
:101370007802FE007908A8007A08A9007B08AA0074
:101380002108031C210FA8022208031C220FA90216
:101390002308031C230FAA027C08AB007D08AC00C5
:1013A000AD01AE017E08AB0728080318280FAC0773
:1013B00029080318290FAD072A0803182A0FAE07BA
:1013C00024082B078312B100831625088312B2006C
:1013D00083162C088A15031CF0292C0FF029F229FA
:1013E0008312B207831626088312B30083162D08D2
:1013F000031CFD292D0FFD29FF298312B307831636
:1014000027088312B40083162E08031C0A2A2E0F05
:101410000A2A08008312B40708007808F9008A1124
:10142000B525B9230800AF01B001B101B201AA018D
:10143000AB01AC01AD01AE01AE1A08000310AA0D5C
:10144000AB0DAC0DAD0DA00DA10DA20DA30DAF0DFB
:10145000B00DB10DB20D27083202031D392A26083E
:101460003102031D392A25083002031D392A2408B8
:101470002F02031C4A2A2408AF022508031C250F4B
:10148000B0022608031C260FB1022708031C270FF1
:10149000B2022A14AE0A1C2A103083120313EF0082
:1014A0001130F0001230F1001330F2001430F3006C
:1014B0001530F4001630F5001730F6001830F7003C
:1014C00030308316850078308600073083129F0005
:1014D00083168113193099002030980080308312D0
:1014E0009800C8010530C900BF01C0011430C10017
:1014F0000830C2000430B1007630B2002530B300AD
:10150000B401C401C301BC01BD010130CA00CB005C
:10151000CC00CD01CE01CF014E30E100E201ED0162
:10152000EB01EC01E301E401E501E601C501D001B5
:10153000EA01C7010130E700E800E900C601013017
:10154000BE008B168B1745086A060319C52A450885
:10155000EA004503031DB62A831698013030850042
:1015600086013030831285008601C52A203083161B
:10157000980030308500783086008312E301E40162
:10158000E501E601C8010530C900C508031D312F7A
:1015900031086302031DD82A32086402031DD82AC9
:1015A00033086502031DD82A3408660203198E2BFE
:1015B0003108E3003208E4003308E5003408E600AF
:1015C0008A118E274408013A8A150319092B023A19
:1015D0000319092B063A0319092B023A0319092B9F
:1015E0000F3A0319092B023A0319092B063A03197A
:1015F000092B083A03190C2B023A03190C2B0F3A4A
:1016000003190C2B023A03190C2B093A03190F2B5F
:10161000182B1F30EE00182B1E30EE00182B033055
:101620003C050319162B1C30EE00182B1D30EE0064
:1016300048038A1103197D2683124308F900FA0131
:10164000FB01FC01790831028316A00083123208E5
:101650008316A100831233088316A2008312340874
:101660008316A3007A08031C7A0FA1027B08031CCF
:101670007B0FA2027C08031C7C0FA3020730A4008E
:10168000A501A601A7018A1513222F08FD00300825
:10169000FE003108A8003208A9000230F8007D08D9
:1016A000F8077808B0000730B1008A1148223408E2
:1016B000F80083126E08F90084273030FA00B12355
:1016C0007808F90084272030FA00B12348038A15EE
:1016D000031D722BED080319722BF9018A1184275F
:1016E0008A15762B4308F9008A1184274030FA00C6
:1016F0008A11B12348038A1503198A2B4808033A33
:1017000003198A2B4808043A03198A2B4808053A1A
:10171000031D8E2B5230FA008A11B1234808003A7B
:101720008A150319AF2B013A0319C72B033A031982
:10173000DB2B013A0319232C073A03195F2C013ADA
:101740000319792C033A0319932C013A0319AE2C8F
:101750000F3A0319C92C013A0319D62CDF2C48087B
:1017600049060319DF2C0530ED004808C9008A112D
:1017700025230030A6002030A5000330A50703185C
:10178000A60A7608A7006A22B9238A15DF2CBE08AC
:10179000031DCC2B0130BE00480849060319DF2C7D
:1017A0004808C9004130E2005230FA008A11B123E2
:1017B0007D268A15DF2CBE08031DE02B0130BE00FC
:1017C000480849060319DF2CC7080319F02B350810
:1017D000B1003608B2003708B3003808B400C701BA
:1017E0001E30ED008A11252383124808C9000030FD
:1017F000F9002030F80020308316A6004130AB00FD
:101800004330A4004530A100A3004630A7004C306F
:10181000A2004D30AA004F30A8005230A90053302A
:10182000A0005430A500AC00AD010030FB00A0309A
:10183000FA005A2641308312E200B9235230FA00EE
:10184000B1238A15DF2C480849060319DF2C1E3006
:10185000ED004808C9006F08F9008A11B52500306D
:10186000AD002030AC000E30AC070318AD0A831277
:101870003C088316A50083123D088316A600643039
:10188000A700A80173233208AE00B1220030F9008E
:101890002030F8000C30F8070318F90A83123C08CE
:1018A0008316A80083123D088316A9006430AA009D
:1018B000AB0192233608FA0072268A15DF2C4808FD
:1018C00049060319DF2C1E30ED004808C9007008D6
:1018D000F9008A11B5250030F9002030F8000E30EB
:1018E000F8070318F90A83124408FA0072268A15C9
:1018F000DF2C480849060319DF2C1E30ED0048088C
:10190000C9007108F9008A11B5250030F9002030AE
:10191000F8000E30F8070318F90A83124308FA009A
:1019200072268A15DF2C480849060319DF2C1E3061
:10193000ED00BE014808C9007208F9008A11B525FA
:101940000030F9002030F8000E30F8070318F90ACB
:1019500083124208FA0072268A15DF2C48084906CD
:101960000319DF2C1E30ED00BE014808C9007308C2
:10197000F9008A11B5250030F9002030F8000E304A
:10198000F8070318F90A83124108FA0072268A152B
:10199000DF2C480849060319DF2C1E30ED004808EB
:1019A000C9007408F8000D228A15DF2C4808490682
:1019B0000319DF2C4808C9007508F8000D228312AE
:1019C00048038A15031DFC2C4608033A0319F42C1E
:1019D0004608043A0319F42C4608063A0319F42C75
:1019E0004608073A031DFC2C410862060319FC2C2B
:1019F0004108E2008A117D2683124808093A8A15B7
:101A00000319102DCA0803190B2DCB0803190B2D30
:101A1000CC08031D102DED080319102D1E30ED000C
:101A20006D08003C03182F2D4808093A03192F2D83
:101A30004008610603192F2D4008E100ED03031D46
:101A40002F2DC70803192D2D3508B1003608B20017
:101A50003708B3003808B400C7010130C8004A088D
:101A6000690603192A2E4A08E900CA08031D2A2E0E
:101A70004808083A0319552D0D3A0319632D063A03
:101A80000319742D073A0319AB2D023A0319CB2D14
:101A9000013A0319DE2D053A0319F12D033A031912
:101AA000FC2D083A03191D2E2A2EC801BF01C001C2
:101AB000C1010B30C200FF30B1007530B2002530DB
:101AC000B300B4012A2EC30A3D218A118E270030AB
:101AD000F9002030F8000E30F8070318F90A43081F
:101AE000FA0072268A152A2EBC0A0319BD0A3D2166
:101AF0008A118E2700308316AD002030AC000E30E6
:101B0000AC070318AD0A83123C088316A5008312A4
:101B10003D088316A6006430A700A801732332088D
:101B2000AE00B1220030F9002030F8000C30F80788
:101B30000318F90A83123C088316A80083123D0893
:101B40008316A9006430AA00AB0192233608FA007C
:101B500072268A152A2E0C30440203182A2E440AB3
:101B6000C4004408023A031DBB2D43081C3C031863
:101B7000BB2D1C30C3003D218A118E270030F90097
:101B80002030F8000E30F8070318F90A4408FA006C
:101B900072268A152A2EC20A4208173C031CC2016B
:101BA0000030F9002030F8000E30F8070318F90A69
:101BB0004208FA008A1172268A152A2EC10A4108A3
:101BC0003B3C031CC1010030F9002030F8000E300E
:101BD000F8070318F90A4108FA008A1172268A15D3
:101BE0002A2E073046020318F72DC60AF82DC60123
:101BF0008A117D268A152A2EC708031D0D2E013055
:101C0000C7001E30ED003108B5003208B6003308B9
:101C1000B7003408B8000130C3000C304402031888
:101C2000132EC40A182E0130C400BC0A0319BD0AC1
:101C30003D218A118E278A152A2E5330FA008A11E7
:101C4000B12300308316A6002030A5007708A70036
:101C50006A22B92383124B0867068A1503191F2FBE
:101C60004B08E700CB08031D1F2F4808053A03194E
:101C70004F2E063A0319642E073A0319A42E023A8E
:101C80000319C32E013A0319D82E053A0319ED2E74
:101C9000033A0319F92E083A03191B2F1F2F430883
:101CA000013C03181F2FC3033D218A118E270030EA
:101CB000F9002030F8000E30F8070318F90A43083D
:101CC000FA0072268A151F2F3D08073C031D6A2E55
:101CD0003C08D03C03181F2FBC080319BD03BC03EC
:101CE0003D218A118E2700308316AD002030AC00D4
:101CF0000E30AC070318AD0A83123C088316A5000A
:101D000083123D088316A6006430A700A801732340
:101D10003208AE00B1220030F9002030F8000C305B
:101D2000F8070318F90A83123C088316A8008312E7
:101D30003D088316A9006430AA00AB01922336083F
:101D4000FA0072268A151F2F4408013C03181F2F22
:101D5000C4034408023A031DB32E43081C3C031875
:101D6000B32E1C30C3003D218A118E270030F900AC
:101D70002030F8000E30F8070318F90A4408FA007A
:101D800072268A151F2FC208031DC92E1730C200E4
:101D9000CA2EC2030030F9002030F8000E30F807D8
:101DA0000318F90A4208FA008A1172268A151F2FB1
:101DB000C108031DDE2E3B30C100DF2EC103003001
:101DC000F9002030F8000E30F8070318F90A41082E
:101DD000FA008A1172268A151F2F4608003C031844
:101DE000F32EC603F52E0730C6008A117D268A150C
:101DF0001F2FC708031D0A2F0130C7001E30ED003A
:101E00003108B5003208B6003308B7003408B8000E
:101E10000130C3004408013C0318102FC403162FDF
:101E20000C30C400BC080319BD03BC033D218A115A
:101E30008E278A151F2F5430FA008A11B12383127E
:101E40004C0868068A150319312F4C08E800CC08A5
:101E5000031D312FC80A0A304802031C312F0130FC
:101E6000C8003230F8008A1105228A15A32A0030F2
:101E700083120313D1000130D2000230D3000330AB
:101E8000D4000430D5000530D6000630D700073026
:101E9000D8000830D9000930DA000A30DB000B30F6
:101EA000DC000C30DD000D30DE000E30DF000F30C6
:101EB000E0008A150A124C2A83120313BF0A3F0856
:101EC0007F3C0318802FBF01C00A40083B3C031829
:101ED000802FC001BE080319802FC10A41083B3C76
:101EE0000318802FC101C20A4208173C0318802F33
:101EF000C201B10A0319B20A0319B30A0319B40AD9
:101F0000061E902FCA08031D9C2F03304D02031C90
:101F10008B2FCD1F8D2FCD0A9C2F0130CA009C2FF7
:101F20004A03031D9C2F4D08003C03189B2FCD1B1B
:101F30009B2FCD039C2FCA01861DAC2FCB08031D00
:101F4000B82F03304E02031CA72FCE1FA92FCE0A95
:101F5000B82F0130CB00B82F4B03031DB82F4E080C
:101F6000003C0318B72FCE1BB72FCE03B82FCB01E1
:101F7000861EC82FCC08031DD42F03304F02031C2C
:101F8000C32FCF1FC52FCF0AD42F0130CC00D42FA1
:101F90004C03031DD42F4F08003C0318D32FCF1B35
:101FA000D32FCF03D42FCC01851EE32F4503031D70
:101FB000F02F03305002031CDF2FD01FE12FD00A77
:101FC000F02FC501F02FC508031DF02F5008003C6D
:101FD0000318EE2FD01BEE2FD003F02F0130C500D9
:101FE0000B113B0E84003A0E8A00390E8300FF0E5F
:041FF0007F0E090057
:02400E00183F59
:00000001FF
